:1000000000308A00E1280000831A0A28A500030EA8
:10001000A6000F288312A500030EA600A6140A0846
:10002000AD008A018313A50E0408A7002008A800CC
:100030002108A9002208AA002308AB002408AC006C
:1000400083128C308400001C27280C18CA2827082B
:1000500084002808A0002908A1002A08A2002B0873
:10006000A3002C08A4002D088A00260E830083120A
:10007000250EA618831609002030D300CF01D00129
:10008000D101D2014A08A3004908A2004808A100F2
:100090004708A0000310201C5B284B08CF074C0822
:1000A00003184C0FD0074D0803184D0FD1074E0809
:1000B00003184E0FD207D20CD10CD00CCF0CA30CCE
:1000C000A20CA10CA00CD30B4A280034A101A20160
:1000D000A001A3014D08031D70284C0803198A28AC
:1000E0001030CE000310CA0DCB0DA00DA30D4D088E
:1000F0002302031D7D284C082002031C86284C087F
:10010000A002031CA3034D08A3020314A10DA20D1A
:10011000CE0B7228000000343308CA003208C90030
:100120003108C8003008C7004130CE00C630CD00CD
:100130004E30CC006D30CB003C2039302007B00071
:100140002108B100303003183130B1072208B20065
:10015000003003180130B2072308B3000030031841
:100160000130B3073208A0003308A100A201A301A7
:100170003308C9003208C8003308CB003208CA006F
:100180007F30CD00FF30CC0066202008A10023087E
:10019000A20000348C202208C8002108C7002208D1
:1001A000CB002108CA000330CD00E830CC00662027
:1001B0002008C6008F0146088E0034140C108A11E6
:1001C000272884011F308305713083168F00831226
:1001D0001F1383161F109F101F119F1107308312CA
:1001E0009900AF010130B000B101B201B301341088
:1001F000B701B80183160108C73908388100853076
:10020000831290000030A10006389200FF30831660
:1002100092000511831205110C30950083160C1401
:10022000C03083128B04713083168F008312341C0C
:100230003A29AE018B1BAE178B138C20AE1B8B178C
:100240002208B8002108B7000330B8053808A2001A
:100250003708A100A20CA10CA20CA10CA20C210831
:100260009300A20C220C3039A0001508CF392004CD
:1002700095003410B70A0319B80A3808A2003708E5
:10028000A100A20CA10CA20CA10CA20C21089300AD
:10029000A20C220C3039A0001508CF39200495009B
:1002A000AE018B1BAE178B138C20AE1B8B17220855
:1002B000B6002108B500AE018B1BAE178B138C2046
:1002C000AE1B8B172208BA002108B900AE018B1BA8
:1002D000AE178B132208CB002108CA00CD01643071
:1002E000CC006620AE1B8B172008B5002308B60093
:1002F000B608031D7F293508623C03188629851539
:10030000831685110511043083128506B608031D76
:1003100091293508013C031C91298511831685110B
:08032000831283161629630005
:02400E00F43488
:00000001FF
